:100000000C94EB060C9413070C9413070C94130731
:100010000C9413070C9413070C9413070C941307F8
:100020000C9413070C9413070C9413070C9453327D
:100030000C9413070C9413070C9413070C941307D8
:100040000C94CF320C9413070C9413070C941307E1
:100050000C9413070C9413070C9413070C941307B8
:100060000C941C220C94130705A84CCDB2D44EB9A5
:100070003836A9020C50B9918688083CA6AAAA2A4B
:10008000BE000000803F50726573732041006174B0
:1000900020747261636B20002E20506C61636500D8
:1000A000596F7520726561636865642000436F6EE7
:1000B00067726174756C6174696F6E73212000548E
:1000C0007261636B206C6F636B6564002F00204C62
:1000D0003A0020506F733A005370643A004C454622
:1000E000540052494748540063757272656E74201B
:1000F0004469723A200070726573732043207768F8
:10010000656E20646F6E65007475726E207269672B
:1001100068742B7072657373205249474854007499
:1001200075726E206C6566742B7072657373204CEB
:10013000454654004144584C3334352063616C6962
:1001400062726174696F6E001573656C656374200B
:1001500016636C65617220176261636B002D2D3A26
:100160002D2D202D2D00200030003A0030002000E1
:10017000100020547261636B202020202020205426
:10018000696D6520506F7300636F756C64206E6FCE
:1001900074206F70656E204441542066696C650060
:1001A000422D52616C6C79000002FA01F201EA0101
:1001B000E401DE01D601CE01C501BC0148617264D3
:1001C000657374320048617264657374310048610C
:1001D0007264657232004861726465723100486110
:1001E000726432004861726431004D656469756DF6
:1001F00032004D656469756D310045617379320077
:1002000045617379310042023A022D022802180238
:1002100042023A022D02280243616C6962726174E3
:100220006520416363656C00457869740053656CB3
:1002300065637420747261636B00526573746172DC
:100240007400526573756D65001010FFFF800187A3
:10025000E187F18071807183E183E1807180718039
:100260007187F187C180018001FFFF1010FFFF80BF
:100270000187C187E184E180E181E183E187C18772
:10028000818E018FE18FE180018001FFFF1010FF5F
:10029000FF800180C187C187C185C181C181C181C2
:1002A000C181C181C181C181C180018001FFFF1075
:1002B0001000003C1E3C3C3C3C1E3C1E381E780E90
:1002C000780F700F7007F007E007E007E003C00049
:1002D00000101000001FE01FF81FF81E7C1E781E83
:1002E000781FF01FE01FF01EF81E781E781E7C1E7F
:1002F0003C00001010000007E00FF81FFC3E7C3CA3
:100300003C3C3E7C1E7C1E3C3E3C3C3FFC1FF80FB0
:10031000F003C0000010100000FC3FFC3FFE3FEE69
:100320003FEE7FEE7FEF7FEF6FE7EFE7EFE7EFE77F
:10033000CFE3CFE3CF00001010000003F80FF81F49
:10034000F83F083E003C003CFC3CFC3CFC3E3C3F93
:100350003C1FFC0FFC03F00000101000000FF00F1A
:10036000F00FF00FF00F000F000FF00FF00FF00F75
:10037000000F000FF80FF80FF80000101000000336
:10038000E007E007E007F00FF00F700E781E781F0F
:10039000F81FFC3FFC3C3C3C3E7C1E000000010280
:1003A00003040505060607070808090909090A0ADA
:1003B0000A0A0A0A0A0A0B0B0B0B0B0B0B0B0C0C91
:1003C0000C0C0C0C0C0C0D0D0D0D0D0D0D0D0E0E61
:1003D0000E0E0E0E0E0E0F0F0F0F0F0F0F0F090642
:1003E0000D01080F01050B0F0104090C0F00030597
:1003F000070B0E0F01030507090B0D0F0001030585
:1004000007090B0D0F0002030506080A0C0D0F006B
:100410000103040607090B0C0E0F00010304050776
:1004200008090B0C0E0F00010204050607080A0B51
:100430000D0E0F0001020304060708090A0C0D0E39
:100440000F0001020304050607090A0B0C0D0E0F2D
:10045000000102030405060708090A0B0C0D0E0F24
:100460001010F0F0F0F0F0F0F0F00F0F0F0F0F0F92
:100470000F0FF0F0F0F0F0F0F0F00F0F0F0F0F0F84
:100480000F0F10107FFEFFFFE007C663C663C66351
:10049000C663CE73CC33D81BD81BD81BC003E00770
:1004A000FFFF7FFE10107FFEFFFFC007CC03CF03CE
:1004B000C3C3C0F3C03BC03BC0F3C3C3CF03CC0333
:1004C000E007FFFF7FFE10107FFEFFFFE007C03355
:1004D000C0F3C3C3CF03DC03DC03CF03C3C3C0F348
:1004E000C033E003FFFF7FFEFFC000FFE000FFE03E
:1004F00000FFF000FFF000FFF800FFF800FFFC0035
:10050000FFFC00FFFE00FFFE00FFFF00FFFFC0FF3B
:10051000FE70FFFE18FFFE18FFFE0CFFFE30FFFC12
:10052000C0FFFCC0FFFD80FFF300FFEC00FFEC000C
:10053000FFB800FE6000FDC000FDC000FB0000F73A
:100540008000EF8000EF8000FFC000FFC000FFE0F0
:1005500000FFE000FFE000FFF000FFE800FFE40024
:10056000FFE400FFC400FFD800FFB000FFB000FFB1
:100570006000FEC000FD8000FD8000F30000E6008A
:1005800000EF0000EF0000FF8000FF8000FFC000D0
:10059000FFC000FFC000FFE000FFF000FFF000FF21
:1005A000F000FFF800FFFC00FFFE00FFFE00FFFD73
:1005B00080FFFC40FFF860FFF860FFC180FE3E0056
:1005C000FFE000FFE000FFC000FFE000FFF000FFE1
:1005D000D800FFD800FFB000FF6000FEC000FF8021
:1005E00000FF0000FE0000FC0000F80000F8000022
:1005F000F80000F80000FF0000FD0000FF8000FF91
:100600008020F800A0FE0020FE0040F80060FC0002
:1006100010FC00A0FFE040FEA020FFC040FC00A8AE
:10062000FFA000FC1010FFC000FFC400F80000FF96
:10063000F280FAB040FFC080FFC040F800C0FF0069
:1006400020FD0080FF0040F80080FC0020FC0080BE
:10065000FE0160FE0000FE0000FE0000FF0000FF43
:100660008000FFC000FFC000101001C00220022067
:1006700001E00020022001C000000FF0B81D700E44
:10068000FFFFFFFFFFFF781E700E101003C0042055
:10069000042003C00420042003C000000FF0B81D94
:1006A000700EFFFFFFFFFFFF781E700E101003C0DB
:1006B00000400040008001000100010000000FF038
:1006C000B81D700EFFFFFFFFFFFF781E700E1010A9
:1006D00001800240020003800240024001800000CD
:1006E0000FF0B81D700EFFFFFFFFFFFF781E700EAA
:1006F000101003C00200038000400040024001804F
:1007000000000FF0B81D700EFFFFFFFFFFFF781E07
:10071000700E10100080010001000200028003C072
:10072000008000000FF0B81D700EFFFFFFFFFFFFFD
:10073000781E700E101001800240004000800040C2
:100740000240018000000FF0B81D700EFFFFFFFF98
:10075000FFFF781E700E10100180024000400080E4
:100760000100020003C000000FF0B81D700EFFFF73
:10077000FFFFFFFF781E700E1010026006900A90B7
:10078000029002900290026000000FF0B81D700EFF
:10079000FFFFFFFFFFFF781E700E1010008001802A
:1007A0000280008000800080008000000FF0B81DF3
:1007B000700EFFFFFFFFFFFF781E700EFFFFFFFFB1
:1007C000F3FFC00FC003C0018001800180018001E0
:1007D0008001800000000000000000000000000117
:1007E00000018001F803FC0FFFFFFFFF0000000085
:1007F000040032F030BC3A3C743E7A3C743E693EB0
:10080000743E603EE43DE0BEC0BDE0FDC0F9C0E620
:10081000F11E7EBE055C02B000000000000000007A
:10082000080031F03AB8303C7A3C743E6A3C753E80
:10083000683E643FE03EE8BDE0BDC0FDC0F9E04673
:10084000F0BE7D5E04BC035000000000FFFFFFFF10
:10085000FC0FF8038001000100010000000000000F
:100860000000000080008001800180018001800183
:10087000C001C003C00FF3FFFFFFFFFF0000000037
:1008800002B0055C7EBEF11EC0E6C0F9E0FDC0BD51
:10089000E0BEE43D603E743E693E743E7A3C743E88
:1008A0003A3C30BC32F004000000000000000000C0
:1008B000035004BC7D5EF0BEE046C0F9C0FDE0BD63
:1008C000E8BDE03E643F683E753E6A3C743E7A3C5B
:1008D000303C3AB831F0080000000000FFFFFBFF99
:1008E000E00FC003C003C0018001800180018001CE
:1008F0000000000000000000000000008001F00186
:10090000F801FC01FE03FE07FF9FFFFF000004004B
:1009100018B03A383878367E7C7E6C7C607C4178C2
:10092000C179C1F9C1F1C1E1C25DF8BD7D7C0ABEEA
:10093000057E03BE01DC01E8006000000000040049
:1009400018B03A38343C3C7E747E687C6478417CD4
:10095000C179C1F9C1F1C1E3E02DF95D7EBC0D7E25
:1009600006BE035E01FC01F800600000FFFFFF9F70
:10097000FE07FE03FC01F801F00180010000000009
:100980000000000000000000800180018001800163
:10099000C001C003C003E00FFBFFFFFF00000060C9
:1009A00001E801DC03BE057E0ABE7D7CF8BDC25DA8
:1009B000C1E1C1F1C1F9C1794178607C6C7C7C7E78
:1009C000367E38783A3818B0040000000000006025
:1009D00001F801FC035E06BE0D7E7EBCF95DE02DD4
:1009E000C1E3C1F1C1F9C179417C6478687C747E4E
:1009F0003C7E343C3A3818B004000000FFFFFFFF93
:100A0000E3FF003F000F00030001000000000000B2
:100A100000000000000000000000000000010003D2
:100A2000000F003FE3FFFFFFFFFFFFFF000000009C
:100A30001C00F5C0E1B0D5F8E27EDC7CD87DCC7C32
:100A4000D87DDA7CC8FDD87CD8FDC87CC07EC1F8D2
:100A5000C1B0E1C01C000000000000000000000068
:100A60001C00EBC0D1F0C37CD57CE87DDC7CD87D5C
:100A7000D87CCAFDC07CDCFDC87CD0FDC17CC97CB3
:100A8000C1F0E1C01C000000000000000A4E6F2011
:100A900053442063617264206F720A6E6F204C4F62
:100AA000414445522E4845580A0A153A457869741A
:100AB000001D20466C617368696E670A20206C6FA8
:100AC000616465722E2E2E0A0A444F4E275420541C
:100AD00055524E204F464621000A0A153A49676E84
:100AE0006F7265006D560A0A504C454153452054BB
:100AF00055524E204F464620004C4F5720424154FD
:100B000054455259212000172B152010204C4F41DD
:100B100044455200172B1620131400175344001697
:100B2000137800161314001510200015201000541F
:100B30000A03E181867F3E186D830F0F0E018386C5
:100B40006033186DC3198F1803C38E6033186DE3BB
:100B500030CF1803C39E603630CDE360CF3006C778
:100B60009E7E3E30CDB360CF300CC6F6603330D9B8
:100B7000B660CF33CFCCF66061B0DB1E60CF30D82B
:100B80006CE6C061B0DB1E618F19986CC6C063B1A2
:100B90009B0E330F0FB078C6FF7E1F1B061E0F057E
:100BA0000089300802380249786814000003053FC4
:100BB000213F1208120A100A0E1C0E0C1E0C141AE9
:100BC00014161F161E131E1E1B1E1E1F1E3F213F26
:100BD0003A2F3A173D173F213F181F02040A041FFE
:100BE0000E04040E1F0A1F0A0E0E1F04110E2E25DE
:100BF0002E2F2A2E262929021F02081F08150E044F
:100C0000040E150E15151B151B040604040C040018
:100C100000000017000300031F0A1F16371A1904EB
:100C2000130A153A000300000E11110E000A040AFF
:100C3000040E040030000404040010001804031F14
:100C4000111F121F101D151711151F07041F17154F
:100C50001D1F151D01011F1F151F17151F000A005D
:100C6000003200040A110A0A0A110A040115020ED0
:100C700011171E051E1F150A0E110A1F110E1F1532
:100C8000111F05010E111D1F041F111F1108100F48
:100C90001F041B1F10101F061F1E040F0E110E1F16
:100CA00009060E112E1F051A121509011F011F102A
:100CB0001F0F180F1F0C1F1B041B031C03191513F8
:100CC000001F11030418111F000201022020200040
:100CD00001020C121E1F120C0C12120C121F0C1A05
:100CE00014041E05242A1E1F021C141D1020201D82
:100CF0001F0814111F101E041E1E021C0C120C3E95
:100D00000A040C123E1E040214160A020F120E10E0
:100D10001E0E100E1E081E120C1226281E322A2627
:100D2000041E21001F00211E040102013F213FF685
:100D3000E8DBCFC3B8AEA49B928A827B746E6862F4
:100D40005C57524E4945413E3A3734312E2C2927C3
:100D500025232145006801000005006801380100D5
:100D6000000500380168010000710D6D0D0101FFE3
:100D7000030101F703000000080002010000030462
:100D800007000000000000000001020408102040DD
:100D90008001020408102001020408102004040449
:100DA0000404040404020202020202030303030314
:100DB0000300000000230026002900000000002599
:100DC0000028002B0000000000240027002A00005B
:100DD0002B11D11F322111241FBECFEFD8E0DEBF6F
:100DE000CDBF11E0A0E0B1E0E6E7F6E702C0059074
:100DF0000D92A23DB107D9F728E0A2EDB1E001C004
:100E00001D92A432B207E1F71DE0C6EDDDE004C09B
:100E10002297FE010E94C739C03DD107C9F70E9441
:100E2000A6360C94393B0C9400008FEF8EBD0DB4A8
:100E300007FEFDCF8EB508958EBD0DB407FEFDCF24
:100E400008950C94233B0C942B3BDC01643508F093
:100E500053C0403308F050C090968C919097342F37
:100E6000359535953595E62FFF27E7FDF095242F2D
:100E70002770823099F4DF01A05FB94F84E5380212
:100E8000A00DB11D11248C9190E0022E02C0959509
:100E900087950A94E2F78095817009C0833039F410
:100EA00046271C968C91482740FF03C014C081112F
:100EB00012C084E53802E00DF11D1124E05FF94F06
:100EC00081E090E0022E01C0880F0A94EAF7809535
:100ED0009081982310C084E53802E00DF11D1124A3
:100EE000E05FF94F81E090E0022E01C0880F0A9484
:100EF000EAF79081982B90830895CF92DF92EF923A
:100F0000FF926B017C012CE137E045E157E06AE09C
:100F100070E088E195E00E94A51F83E891E00E94BF
:100F2000DC1C892B41F4C701B601FF90EF90DF90E4
:100F3000CF900C942B1E48EC68E871E08FE794E0AA
:100F4000FF90EF90DF90CF900C944923CF93DF93E5
:100F500000D000D000D0CDB7DEB745EF51E064E05F
:100F600070E087EF91E00E942B1D9093F401809335
:100F7000F301892B51F16091DA0170E080E090E09B
:100F800021E1660F771F881F991F2A95D1F72091BD
:100F9000EA013091EB01220F331F220F331F620F42
:100FA000731F811D911D6C5F7F4F8F4F9F4F0E945C
:100FB0007D0745EF51E064E070E087EF91E00E942B
:100FC0002B1D9093F4018093F3013091F80150911F
:100FD000F9015F5F6091FA012091F70140E070E054
:100FE00080E090E026960FB6F894DEBF0FBECDBF2E
:100FF000DF91CF91089563E570E080E595E00E9470
:10100000B62080E595E00E942F21811103C081E088
:101010008093D7010895CF93DF9362EB80E090E057
:101020000E9423076CEA81E090E00E94230762EEB1
:1010300082E090E00E942307C3E0D0E0CE010E944E
:101040002107882321F060E0CE010E94230721962A
:10105000C11584E0D80791F7DF91CF91089580E022
:1010600090E00E942107823B61F481E090E00E94C1
:1010700021078C3A31F482E090E00E942107823E01
:1010800039F00E940B081092DA0110920F010895B6
:1010900084E090E00E9421078093DA0185E090E0EF
:1010A0000E94210780930F0108958F929F92AF9223
:1010B000BF92CF92DF92EF92FF920F931F93CF9345
:1010C000DF93982E862EEA0180E090E00E942107AF
:1010D000823B61F481E090E00E9421078C3A31F478
:1010E00082E090E00E942107823E71F0DF91CF9173
:1010F0001F910F91FF90EF90DF90CF90BF90AF9036
:101100009F908F900C940B08CE0164E170E00E94D8
:101110004239EB01A92CB12C7501EE0CFF1CEE0C31
:10112000FF1C670136E0C30ED11CC6010E942107D7
:101130008701095F1F4F9701285F3F4F790188237F
:10114000B9F0881620F4682DC6010E942307C80153
:101150000E942107D82EC7010E9421072D2D30E0C3
:10116000322F2227280F311DC217D30768F404C07D
:10117000682DC6010E9423076D2FC8010E94230716
:101180006C2FC7010E9423079092D90123E02815F4
:1011900098F020910E0130E021503109A216B306DB
:1011A0001CF493949092D9018091D90190910F01F0
:1011B000981710F480930F0184E090E00E942107BB
:1011C0006091D901861721F084E090E00E94230706
:1011D00085E090E00E94210760910F01861781F061
:1011E00085E090E0DF91CF911F910F91FF90EF90FC
:1011F000DF90CF90BF90AF909F908F900C9423077B
:10120000DF91CF911F910F91FF90EF90DF90CF90E2
:10121000BF90AF909F908F9008950F931F9341338D
:1012200008F08FC0853591050CF08BC077FD89C023
:10123000342F3770E1E0F0E001C0EE0F3A95EAF7A5
:101240005E2FAE2FA095E42FE695E695E69534E562
:10125000E39FF001112497FF02C080E090E08E0F21
:101260009F1F6535710514F064E570E06E0F7F1FF8
:1012700021110FC0861797070CF063C0E0917D0421
:10128000F0917E04E80FF91F20812A232083019624
:10129000F1CF213079F4861797070CF052C0E09116
:1012A0007D04F0917E04E80FF91F2081252B208317
:1012B0000196F1CF233009F044C00091F004109161
:1012C000F1042091F2043091F304040F111D211D4B
:1012D000311D6150710900FF1AC0861797078CF500
:1012E000E0917D04F0917E04E80FF91F2081252B09
:1012F000208302969C0121503109E0917D04F091F8
:101300007E04E20FF31F20812A232083E6CF861775
:101310009707BCF4E0917D04F0917E04E80FF91F7B
:1013200020812A23208302969C0121503109E091DB
:101330007D04F0917E04E20FF31F2081252B208392
:10134000E6CF1F910F9108952F923F924F925F9297
:101350006F927F928F929F92AF92BF92CF92DF92C5
:10136000EF92FF920F931F93CF93DF9300D01F92C2
:10137000CDB7DEB741504F3008F090C0853508F04A
:101380008DC0613308F08AC0480152E0850E911C7F
:1013900030E050E00FE010E03801641A750A5A019D
:1013A000AA0CBB1CA501475D5E4F5B834A83262EBA
:1013B000312C90E0EE24E394F12C632F70E066155D
:1013C00077050CF06BC0EA81FB81C080D180F6010B
:1013D000E60FF71F4491F401E40FF11DE40FF11D36
:1013E000B4903196A490DB01A20DB31DAD01F3E0E2
:1013F00055954795FA95E1F7473009F44DC0F4E566
:10140000F49FB001F59F700D1124680F791F605F84
:10141000794FA770BB27A70102C0440F551FAA959B
:10142000E2F7DA0149834B2D50E0542F44274A0D4F
:10143000511D512C4A2E4094A52DB0E0A615B7059C
:101440005CF5F601EA0FFB1FE4915D01A80EB91EE1
:10145000F4E5AF16B104F4F45801AE1AB108F50181
:10146000570102C0AA0CBB1CEA95E2F7F501A422C1
:10147000B522AE16BF0639F4A60FB71FBC90A980DF
:10148000BA28BC9207C0222329F0A60FB71FEC91FF
:10149000E421EC935394D0CF3F5F8FCF0F900F9008
:1014A0000F90DF91CF911F910F91FF90EF90DF9000
:1014B000CF90BF90AF909F908F907F906F905F90F4
:1014C0004F903F902F90089520E030E09FEF87FDF0
:1014D000805863E08602A0011124FA01E651FB4F17
:1014E000E491A0917D04B0917E04A20FB31FEC9310
:1014F000FA01E751FB4FE49160917D0470917E0405
:10150000620F731FDB01AC5ABF4FEC93FA01E85135
:10151000FB4F449160917D0470917E04620F731FB4
:10152000FB01E855FF4F408340917D0450917E04BC
:10153000420F531FFA01E450FF4F908340917D0406
:1015400050917E04420F531FFA01E05BFE4F9083DF
:101550008F5F2F5F3F4F2435310509F0B8CF0895D5
:10156000EF92FF920F931F93CF93DF93992787FDFD
:10157000909582599E4FC0917D04D0917E04C80FF2
:10158000D91FDE01AC5ABF4F80E090E070E0660FDB
:10159000771FAB01435A5E4F8B010B581E4F6759A3
:1015A0007E4FFA0120813181280F391FF9013491D2
:1015B0002C9123232C939C012F5F3F4FFA01E08055
:1015C000F180E20EF31EF701E490F881FE21F8832A
:1015D000E091F004E0FF02C0FB0101C0F801E080EF
:1015E000F180E80EF91EF701E490FC91FE29FC93CE
:1015F000E091F004E0FF02C0FB0101C0F801E080CF
:10160000F180E20EF31EF701E49028812E29299340
:10161000029611968033910509F0C3CFDF91CF91E7
:101620001F910F91FF90EF900895CF93E82F809135
:10163000F00480FD02C0FAEA01C0F5E5CF2FC095A5
:1016400080E390E08E1B9109E7FD939568E070E0E0
:101650000E945639682FE7FDE95FE595E595E59528
:10166000611101C0E15091E09E0F9630ACF424E589
:101670009202A0011124405F594F20E030E0DA01CE
:10168000A20FB31FFC931196CC932E5F3F4F2435CE
:101690003105A9F79F5FE9CF662341F147E050E0AC
:1016A000481B510987FD539521E030E0042E01C00D
:1016B000220F0A94EAF721953F2F3223C223209567
:1016C00084E5E89FF0011124E05FF94FDF011196F6
:1016D00090E080818223832B80838C9182238C2BCA
:1016E0008C939E5F32961296943599F7CF91089518
:1016F0000F931F93CF93DF93C091F201D6E0CC23D9
:10170000A1F08C2F90E00197D89FF001D99FF00DA8
:101710001124E15AFD4F00811181258143816481AB
:1017200082810E94A409C150EACFDF91CF911F911D
:101730000F91089568ED70E08DEC94E00E943835CB
:101740004AE050E0609111018DEC94E00E943A363D
:1017500062ED70E08DEC94E00E9438354AE050E094
:101760006091DF018DEC94E00E943A366EEC70E0FF
:101770008DEC94E00E9438358091EA019091EB0164
:101780008654910960910A0170910B010E944239BF
:1017900077276F5F7F4F4AE050E08DEC94E00E9426
:1017A00025366CEC70E08DEC94E00E943835809129
:1017B0000C0190910D0160910A0170910B010E9442
:1017C00042394AE050E08DEC94E00C943A36EF92C6
:1017D000FF920F931F93CF93DF938C01EB01F42EB5
:1017E000E22E01978E379105A0F461E0261360E0A8
:1017F0008DEC94E00E94E52A4F2D6FEF600F8DEC89
:1018000094E00E9425074F2D602F8DEC94E00E94FC
:10181000250760E08DEC94E00E94E52A0F37110562
:101820002CF5C2388FEFD807D4F461E0E61260E0FF
:101830008DEC94E00E94E52A4F2D6C2F8DEC94E006
:101840000E9425076C2F6F5F4F2D8DEC94E0DF9188
:10185000CF911F910F91FF90EF900C94250720E0FE
:101860004F2DBE01C80101960E940D09C435D10556
:10187000E4F2DF91CF911F910F91FF90EF900895C7
:101880000F939091F201953178F456E0959FF00115
:101890001124E15AFD4F8383628344833183208383
:1018A00005839F5F9093F2010F9108957F928F922D
:1018B0009F92AF92BF92CF92DF92EF92FF920F93DF
:1018C0001F93CF93DF931092EB011092EA011092D5
:1018D000E1011092ED011092EC0110921101609162
:1018E000DA0170E080E090E0E1E1660F771F881F89
:1018F000991FEA95D1F70E942B1E45EF51E062E057
:1019000070E087EF91E00E942B1D9093F40180938B
:10191000F3018091F70190E0982F88272091F8013A
:10192000820F911D90930D0180930C0145EF51E0C2
:1019300062E070E087EF91E00E942B1D9093F4012C
:101940008093F3018091F70190E0982F88272091F0
:10195000F801820F911D90930B0180930A0100E022
:1019600010E0B6E0FB2EF09EE001F19ED00D1124B8
:10197000C952DD4F0E94A607288339834A835B83BF
:101980006C837D838091EA019091EB0101969093A5
:10199000EB018093EA010F5F1F4F0634110519F721
:1019A0000BEF11E087E4A82E81E0B82E94E0E92E39
:1019B00092E0F92E24E5C22E23E0D22ECBE0D0E037
:1019C0003BE0732E4EE1842E5CE0952E672D6C1B60
:1019D000F801D383C283F501819191915F01F801F0
:1019E00091838083F7013597862F8170889D802DA4
:1019F00011248F50808370E080E090E00E94B23725
:101A000020E030E040E251E40E941E379B01AC012F
:101A100060E070E080E090E40E94B636F8016583F3
:101A2000768387839087F7011082892D8C1BF601BE
:101A300080832197065F1F4FFAE0EF0EF11C86E0CE
:101A4000C81AD108C130D10509F68BE08093DF01B7
:101A50001092DE011092DD018CE38093DB0183E0C4
:101A60008093DC01E091DA01F0E0EE0FFF1FE85512
:101A7000FE4F659174914CE38FE794E0DF91CF9135
:101A80001F910F91FF90EF90DF90CF90BF90AF909C
:101A90009F908F907F900C94492390910F019817FD
:101AA00038F44CE36FEB70E08FE794E00C9449233B
:101AB0008093DA010C94560C7F928F929F92AF9292
:101AC000BF92CF92DF92EF92FF920F931F93CF932B
:101AD000DF93CDB7DEB72C970FB6F894DEBF0FBEFD
:101AE000CDBF80E090E00E942107823B61F481E05D
:101AF00090E00E9421078C3A31F482E090E00E944D
:101B00002107823E19F00E940B08EAC08091D8019B
:101B1000863008F4E3C01BEF180F62E771E08DEC2C
:101B200094E00E946835912EE12EF12C85E0E80EBC
:101B3000F11C33E3832E4CE3A42EB12C092D10E0CD
:101B4000E016F1060CF482C08091D801891103C01F
:101B500060E771E002C06EE671E08DEC94E00E94F7
:101B60003835F801EE0FFF1FE855FE4F659174916F
:101B7000CE0101960E940E3BBE016F5F7F4F8DEC40
:101B800094E00E945B358092D6046801CC0CDD1C89
:101B9000CC0CDD1CC60107960E942107082FC60148
:101BA00008960E94210710E0102F0027080F111D32
:101BB0000115110509F442C0C801B5010E9442395E
:101BC000762E89E0861730F06CE671E08DEC94E0BB
:101BD0000E9438354AE050E0672D8DEC94E00E9479
:101BE0003A366AE671E08DEC94E00E943835C8011F
:101BF000B5010E9442398C018A30910530F468E6C3
:101C000071E08DEC94E00E9438354AE050E0602F9E
:101C10008DEC94E00E943A3666E671E08DEC94E03B
:101C20000E943835C60106960E9421074AE050E01E
:101C3000682F8DEC94E00E94413606C06DE571E09E
:101C40008DEC94E00E946835939478CF68E471E05D
:101C50008DEC94E00E94683566E089E894E00E948B
:101C6000312A882319F081E08093DC0163E089E860
:101C700094E00E94312A882371F04091D801242FEA
:101C800030E080910E0190E00197281739071CF48D
:101C90004F5F4093D80161E089E894E00E94312AC7
:101CA000882339F08091D801882319F081508093DE
:101CB000D80148E265E089E894E00E94432A811156
:101CC0000E940B0864E089E894E00E94312A88238E
:101CD00039F08091D8010E944D0D02C010E01DCF57
:101CE0002C960FB6F894DEBF0FBECDBFDF91CF911B
:101CF0001F910F91FF90EF90DF90CF90BF90AF902A
:101D00009F908F907F9008952F923F924F925F9275
:101D10006F927F928F929F92AF92BF92CF92DF92FB
:101D2000EF92FF920F931F93CF93DF93CDB7DEB760
:101D30002E970FB6F894DEBF0FBECDBFE091DA014B
:101D4000F0E0EE0FFF1FE855FE4F65917491CE0154
:101D500001960E940E3B8091DF01843030F46DEAE1
:101D600070E08DEC94E00E94683560EA70E08DECE4
:101D700094E00E9468354AE050E06091DF018DEC0C
:101D800094E00E943A3668E970E08DEC94E00E949D
:101D900068356EE870E08DEC94E00E943835BE0145
:101DA0006F5F7F4F8DEC94E00E947A3566E870E0BB
:101DB0008DEC94E00E94383589E291E09E878D8712
:101DC000C12CD12C76016091F0047091F1048091C6
:101DD000F2049091F3046C0D7D1D8E1D9F1D0E94D9
:101DE000B2372B013C0120E030E040EA51E40E9490
:101DF0001E370E941B374B015C0120E030E040EFB2
:101E000051E4C301B2010E941E370E94DC381B015D
:101E10002C01ED85FE8512910291FE87ED8720E071
:101E200030E040EE50E4C501B4010E94793820E072
:101E300030E040E051E40E94B7360E948637762EAB
:101E400020E030E040E851E4C501B4010E94793857
:101E50009B01AC0160E070E080E891E40E94B6363E
:101E60000E948637B62E20E030E048E052E4C201FE
:101E7000B1010E94793820E030E048E052E40E944D
:101E8000B7360E948637862F20E0472D6B2D0E94A3
:101E9000A409F8E0CF0ED11CE11CF11C80E4C816A7
:101EA000D104E104F10409F08ECF64E089E894E004
:101EB0000E94312A882331F08091D9018093DA0180
:101EC0000E944D0D2E960FB6F894DEBF0FBECDBF0B
:101ED000DF91CF911F910F91FF90EF90DF90CF9006
:101EE000BF90AF909F908F907F906F905F904F903A
:101EF0003F902F9008952F923F924F925F926F9252
:101F00007F928F929F92AF92BF92CF92DF92EF9289
:101F1000FF920F931F93CF93DF93CDB7DEB72A972E
:101F20000FB6F894DEBF0FBECDBF2091EA0130910D
:101F3000EB013B832A83265431093D832C83609037
:101F40000A0170900B01C901B3010E9442396C0172
:101F50003091DC013E8320900C0130900D0184E132
:101F6000280E311CEDEFF1E0FA87E98704E012E07A
:101F7000E12CF12CFBE0F98396012A5B3F4F388777
:101F80002F8366E0562E4E2C3E81313049F5E9858F
:101F9000FA8520813181C1018E0D9F1D28173907D7
:101FA000F8F4F801608170E080E090E00E94B437BE
:101FB0004B015C0120E030E040EC51E4E985FA851A
:101FC00063817481858196810E9479389B01AC017F
:101FD000C501B4010E94B7360E948637F8016083BC
:101FE000F8018081893180F068E10E943639E98505
:101FF000FA8520813181280F311D31832083F8013A
:1020000080810E9436399083E985FA85A080B1806D
:102010002C813D81A216B30618F4398131503983E1
:10202000C501B3010E944239EF81F8858E179F07E1
:1020300008F040C0C816D906E8F58C199D09589ECD
:10204000F001599EF00D1124E952FD4F808199272E
:1020500087FD909597FF03C0919581959109BC01EB
:10206000882777FD8095982F0E94B43720E030E0D4
:1020700040EE50E40E941E379B01AC0160E070E02E
:1020800080E090E40E94B636E985FA856383748324
:1020900085839683C501B3010E9442398C199D093D
:1020A000589EF001599EF00D1124E952FD4F4394C2
:1020B00045822EC0642D70E080E090E00E94B2372F
:1020C00020E030E040E251E40E941E379B01AC0169
:1020D00060E070E080E090E40E94B636E985FA8521
:1020E0006383748385839683F8ECAF0EB11C2A81D9
:1020F0003B81A216B30660F420E030E040E85FE3E5
:102100000E94B736E985FA85638374838583968355
:10211000FFEFEF1AFF0A29853A85265F3F4F3A877E
:102120002987065F1F4F3AE0E316F10409F02BCF31
:1021300089818093DF012A960FB6F894DEBF0FBE27
:10214000CDBFDF91CF911F910F91FF90EF90DF9066
:10215000CF90BF90AF909F908F907F906F905F9047
:102160004F903F902F9008957F928F929F92AF92C1
:10217000BF92CF92DF92EF92FF920F931F93CF9374
:10218000DF9300910A0110910B018091EA01909177
:10219000EB0186549109B8010E9442397C01C0903C
:1021A000EC01D090ED014091120170901101CFEF40
:1021B000D1E0FE01329780819181B8010E944239BD
:1021C000E816F90680F59701240F311D8217930751
:1021D00050F588819601280F311D87FD3A95C90178
:1021E0000E964D9700F589809A80AB80BC8020E0E8
:1021F00030E040EA51E4C501B4010E9479380E9400
:102200008637762E20E030E040EA50E4C501B40184
:102210000E94793820E030E040EC50E40E941E3704
:102220000E948637462F2A9632E0C336D30709F03C
:10223000C0CF4093120170921101DF91CF911F9195
:102240000F91FF90EF90DF90CF90BF90AF909F9055
:102250008F907F9008951092D0041092CF048CEB51
:1022600091E09093CE048093CD0480E196E090932A
:102270007E0480937D0408951F93CF93DF931F9274
:10228000CDB7DEB7162FBC0180E595E049830E94EB
:10229000B620612F80E595E00E9463204981642F7C
:1022A00080E595E00E94632080E595E00F90DF9146
:1022B000CF911F910C942F2140E06DE283E590E0D7
:1022C0000E943C1140E16DE283E590E00E943C11E8
:1022D0004BE061E383E590E00E943C1148E06DE251
:1022E00083E590E00E943C1146E06CE283E590E0DB
:1022F0000E943C1140E86EE283E590E00E943C11B0
:1023000064E670E080E090E00E94483340E06EE1D7
:1023100083E590E00E943C1140E06FE183E590E0AE
:102320000E943C1140E060E283E590E00C943C1197
:102330008FE794E00E94D02860EA71E08FE794E094
:102340000E9455281092970480E595E00E94A220F3
:102350000E94FB078091D70181110E945C1160E00F
:1023600070E0CB010E947D070E942F080C94560C50
:10237000109211011092EB011092EA010C94981145
:102380008091D701811104C044E060E172E003C094
:1023900045E066E072E08FE794E00E94102582300D
:1023A00079F02CF4882341F0813041F00895833096
:1023B00059F0843059F0089581E009C00C94560C0E
:1023C0001092D80185E003C00C94B81186E0809388
:1023D000DC010895EF92FF920F931F93CF93DF9349
:1023E00000D000D0CDB7DEB77C01162FBC0180E550
:1023F00095E02B833C8349835A830E94B620612F4A
:1024000080E595E00E94632080E595E00E942F2101
:10241000B70180E595E00E94B62049815A81B70155
:1024200080E595E00E942C212B81022F3C81132F07
:1024300080E595E00E940B20892B41F080E595E036
:102440000E941320F80181938F01F2CF80E595E07F
:102450000F900F900F900F90DF91CF911F910F91E0
:10246000FF90EF900C942F210F931F93CF93DF9346
:1024700000D000D000D0CDB7DEB78C019E012F5F19
:102480003F4F46E050E062E383E590E00E94EA11AE
:102490008A8190E0982F88272981822BF8019183E7
:1024A00080838C8190E0982F88272B81822B9383C7
:1024B00082838E8190E0982F88272D81822B9583AF
:1024C000848326960FB6F894DEBF0FBECDBFDF9192
:1024D000CF911F910F910895CF93DF9300D000D03B
:1024E00000D0CDB7DEB764E371E08DEC94E00E94DC
:1024F00068356FE171E08DEC94E00E94683568E02A
:1025000071E08DEC94E00E94683566EF70E08DEC30
:1025100094E00E946835CE0101960E94341266E074
:1025200089E894E00E94312A882319F081E08093A1
:10253000DC0160E089E894E00E94312A882331F0D0
:102540008B819C819093D6018093D50162E089E8CC
:1025500094E00E94312A882331F08B819C819093F2
:10256000D4018093D30141E02091D5013091D6016F
:102570008091D3019091D401821793070CF040E031
:102580004093D20168EE70E08DEC94E00E94383503
:102590004091D2012B813C818091D3019091D40153
:1025A000442331F0821B930B1816190634F00BC02C
:1025B000281B390B1216130634F462EE70E08DEC12
:1025C00094E00E9438354091D2012B813C8180916A
:1025D000D5019091D601442321F0821B930B892FC2
:1025E00003C0281B390B832F881F8827881F31F0D1
:1025F0006DED70E08DEC94E00E94383526960FB6B4
:10260000F894DEBF0FBECDBFDF91CF9108952F921A
:102610003F924F925F926F927F928F929F92AF9272
:10262000BF92CF92DF92EF92FF920F931F93CF93BF
:10263000DF93CDB7DEB729970FB6F894DEBF0FBE94
:10264000CDBF4091DD015091DE014F5F5F4F509350
:10265000DE014093DD0180910C0190910D018A5BB8
:102660009F4F2091EA013091EB018217930768F4A4
:102670008091DC01813049F482E08093DC0160913B
:10268000DF018091DA010E94550841E060E089E8AD
:1026900094E00E94512A882321F08091100181301A
:1026A000E1F541E062E089E894E00E94512A882344
:1026B00021F0809110018530A1F541E065E089E8C5
:1026C00094E00E94512A8823C1F080911101843046
:1026D00020F084508093110102C01092110180916A
:1026E0001001823019F481E0809310018091100173
:1026F000843019F485E08093100141E064E089E8BA
:1027000094E00E94512A20911101882371F0809158
:10271000DC01833009F0BBC308C082E08093100164
:10272000C0CF84E080931001C8CF222319F021503C
:102730002093110162E089E894E00E943A2A8823FC
:1027400029F08091D70181110FC0B0C360E089E802
:1027500094E00E943A2A8111F4CF64E089E894E081
:102760000E943A2A8111EDCF8091D701882309F484
:1027700076C0CE0101960E9434124091D201209180
:10278000D5013091D6018B819C81442319F0281BFF
:10279000390B04C0BC01621B730B9B01232F221F4A
:1027A0002227221F39F020911001213019F022E058
:1027B000209310012091D3013091D401442331F0B2
:1027C000281B390B1216130634F00CC0821B930B16
:1027D000181619063CF480911001853019F084E038
:1027E0008093100162E089E894E00E943A2A811106
:1027F00061C360E089E894E00E943A2A81115AC3DB
:1028000064E089E894E00E943A2A811153C3409120
:10281000D2012091D5013091D6018B819C81442336
:1028200031F0281B390B1216130644F018C0FC01B6
:10283000E21BF30B1E161F0654F011C02091D301AA
:102840003091D401281B390B37FF09C033C32091C5
:10285000D3013091D401821B930B97FD2BC3809140
:1028600010018230A9F018F4813031F03EC084307C
:10287000D9F0853031F139C02091EC013091ED0172
:102880002035310594F58091120190E00A9627C019
:102890002091EC013091ED012035310534F5809126
:1028A000120190E005961BC02091EC013091ED01E2
:1028B000213BFFEF3F07CCF0409112018BEF9FEFE0
:1028C0000CC02091EC013091ED01213B4FEF34071A
:1028D00064F04091120186EF9FEF841B9109820FF3
:1028E000931F9093ED018093EC0166E089E894E0FA
:1028F0000E94312A81111092DC018091EC019091AB
:10290000ED012091DA0262EE6203A0011124841726
:1029100095073CF07EE1279F900111242817390785
:10292000A4F480911101853118F0869580931101EE
:1029300080911101882349F08091E001813011F4E8
:102940008FEF01C081E08093E00183E680937C04F7
:1029500080937B041092F1011092F0011092EF012C
:102960001092EE018091110168E10E943639809346
:1029700012010E94B410F09012012F2D30E08091CE
:10298000EA019091EB01820F931F9093EB018093EA
:10299000EA011092F20160E086E490E0821B930B62
:1029A00076E0462F50E048175907BCF4749FD001D9
:1029B000759FB00D1124A952BD4F420F531F749F34
:1029C000F001759FF00D1124E952FD4F472F019042
:1029D0000D924A95E1F76F5FE4CF76E4C72ED12CD4
:1029E000E6E0EE2EFF20A9F0C6018F199109E89EBE
:1029F0008001E99E100D112409521D4F0E94A60767
:102A0000F801208331834283538364837583FA946E
:102A1000E9CF6091D702709112016703A0011124E0
:102A20002091EC013091ED01240F351F3093ED0121
:102A30002093EC018091E101723028F0962F67FD20
:102A40009F5F959501C090E0980F9093E101809170
:102A5000E001890F0E94640A0E949A0B0091EE0126
:102A60001091EF01D0907B04EFEDF2E021E030E037
:102A700058E1E52EF12C65E0C62EDF0111978C910F
:102A8000080F111D87FD1A95C701B9010E9456391B
:102A900048E1B42EB60EC09EC001C19E900D112417
:102AA000B9016C5F7F4F0E945639B60EB082AB2DD4
:102AB000BB27A7FDB0954D2D50E0A417B5070CF42A
:102AC000DB2C2F5F3F4F369626343105B1F610933D
:102AD000EF010093EE01D0927B048D2D0E94150B27
:102AE0000E947B0F1092E9011092E80184E590E0CA
:102AF0009093E7018093E60192EEA92E92E0B92E21
:102B0000CC24C394D12C33E0232E312CF501339700
:102B100070803196208133978081E090F001F090B1
:102B2000F101E80EF11C87FDFA94F092F101E092B8
:102B3000F001FAE2EF0EF11C8091EC019091ED01B1
:102B4000B6010E945639E60EF71E3EE1239FC001F2
:102B50001124B6010E9456397727C701861B970BAF
:102B60009093E5018093E4016E0D7F1D7093E30166
:102B70006093E20180917C04781608F070C045E013
:102B8000471508F06CC0682E671800E010E0862C2E
:102B9000912CE091E201F091E3012091E401309168
:102BA000E501061508F051C08091EA019091EB0112
:102BB0008C0D9D1DB1010E944239CB01B1010E94D3
:102BC00042398F83472D400FE09FC001E19F900D58
:102BD000F09F900D1124B4010E945639E61BF70BAB
:102BE0006091E6017091E701069FC001079F900D7B
:102BF000169F900D1124B4010E945639E60FF71F5D
:102C0000209FC001219F900D309F900D1124B40191
:102C10000E9456392901461A570A2091E80130913D
:102C2000E901029FC001039F900D129F900D112496
:102C3000B4010E945639CB012F81BF01840D951D2F
:102C40000E94E70B0F5F1F4FA4CF3093E901209341
:102C5000E801F093E701E093E60170927C04809133
:102C6000F201843108F0C8C05FE35C1508F4C4C009
:102C7000F601E356FC4F149180E1682E611A572C3F
:102C80005618F501319780818230B1F120F48130FE
:102C900009F445C081C0833009F454C0853009F07F
:102CA0007BC0862D880F5E2D581B862D67FE02C0C7
:102CB00081E0860D8595581B90E004E0402E470189
:102CC000810E911C711A1E141F048CF464E5861683
:102CD00091046CF401E020E634E0472D692F650F84
:102CE000812F598798870E94400C988559854A946E
:102CF000960D4110E8CF50C06091E2017091E30160
:102D0000CB01810F911D843591050CF045C016163D
:102D100017060CF041C001E026EC34E039C06091A8
:102D2000E4017091E501862D992787FD909586171E
:102D3000970794F5643571057CF5661901E024EA7E
:102D400034E026C06091E4017091E501862D992759
:102D500087FD9095861797075CF46435710544F4F8
:102D6000661901E022E834E0452D812F0E94400CD5
:102D70006091E2017091E301CB01810F911D8435D7
:102D8000910554F4161617063CF401E022E834E0ED
:102D9000452D812F0E94400CF5018081882361F12F
:102DA0009091F201943140F51E141F041CF5970117
:102DB000210F311D24353105ECF490E001972AE014
:102DC000289FF001299FF00D1124E550FE4F20812E
:102DD00031818481992787FD9095B6010E945639EB
:102DE0006E0D67FC63946594661900E0452D812F94
:102DF0000E94400CF5011082FFEFCF1ADF0A26E097
:102E0000A20EB11C36E4C316D10409F07FCE0E9495
:102E1000780B609110018091E0010E94B00A6091EE
:102E200011016F7120E041E084EA94E00E94663075
:102E30008091DC01833009F041C08091DB01815039
:102E40008093DB01811104C081E08093DC0136C0F6
:102E500064E10E943639392F3695E82FF0E0EE0F05
:102E6000FF1FED5EFE4F0081118164E0630F21E0E2
:102E7000492F82E2830F0E94A4098091DD01909185
:102E8000DE0101979093DE018093DD0117C02639A2
:102E900008F050CC86E191E0821B9109880F892FC0
:102EA000881F990B820F8093110144CC83E080939B
:102EB00010015ACC83E080931001D1CC29960FB633
:102EC000F894DEBF0FBECDBFDF91CF911F910F9160
:102ED000FF90EF90DF90CF90BF90AF909F908F903A
:102EE0007F906F905F904F903F902F9008958FE765
:102EF00094E00E9403248823D9F08091DC01823081
:102F000069F028F4882361F0813061F008958530FC
:102F100059F0863059F0833059F404C00C94840E73
:102F20000C94C0110C9407130C945C0D0C946C124F
:102F30000895E0910E05F0910F050995E0911205B5
:102F4000F09113050994FF920F931F93CF93DF9392
:102F5000C82FD42F152F062FF72E87FF0AC040E069
:102F600050E0BA0187E70E94A317823008F04DC0F5
:102F7000CF77E0910E05F0910F050995E0911005CE
:102F8000F09111050995E0911205F091130509954D
:102F9000E0911205F091130509958F3FC9F7E09173
:102FA0001405F09115058C2F0995E0911405F09109
:102FB00015058F2D0995E0911405F0911505802FC9
:102FC0000995E0911405F0911505812F0995E0917F
:102FD0001405F09115058D2F0995C03421F0C834E2
:102FE00021F081E003C085E901C087E8E091140584
:102FF000F09115050995CAE0E0911205F0911305CD
:10300000099587FF02C0C150B9F7DF91CF911F9199
:103010000F91FF9008959093150580931405709378
:1030200013056093120550931105409310053093DA
:103030000F0520930E050895EF92FF920F931F93B3
:10304000CF93DF9300D000D01F92CDB7DEB714E648
:10305000E0911205F091130509951150C9F740E070
:1030600050E0BA0180E40E94A317813009F057C0F4
:103070004AEA51E060E070E088E40E94A3178130E2
:1030800039F57E0185E0E80EF11C8E010F5F1F4FC0
:10309000E0911205F09113050995F80181938F01D4
:1030A000EE15FF05A9F78B818130C9F58C818A3A2D
:1030B000B1F508EA11E640E050E060E070E489EE26
:1030C0000E94A3178823A9F101501109A1F727C075
:1030D00040E050E0BA0189EE0E94A317823020F44C
:1030E00092E0F92E99EE03C0FF24F39491E408EAEC
:1030F00011E640E050E0BA01892F9D830E94A3179A
:103100009D81882321F00150110999F708C040E002
:1031100052E060E070E080E50E94A3178111F12C7D
:10312000F0921F080E94991781E0FF2009F180E0CA
:103130001FC040E050E0BA018AE70E94A317811146
:10314000EECF8E010F5F1F4FE0911205F091130536
:103150000995F80181938F01EE15FF05A9F7898183
:1031600086FF03C02CE0F22EDBCF84E0F82ED8CF10
:103170000F900F900F900F900F90DF91CF911F91B4
:103180000F91FF90EF9008958F929F92AF92BF9210
:10319000CF92DF92EF92FF920F931F93CF93DF9323
:1031A0001F92CDB7DEB76C0179014801E89497F81A
:1031B0008114910409F484C0C401820F931F8130EB
:1031C000924008F07DC080911F0883FD07C0E9E0B0
:1031D000440F551F661F771FEA95D1F781E50E94BE
:1031E000A317811165C048EEA42E43E0B42EE091F0
:1031F0001205F091130509958F3F29F481E0A81A73
:10320000B108A9F755C08E3F09F052C032E0A32E95
:10321000BA2CAE18BF08A818B908E114F10449F097
:10322000E0911205F0911305099591E0E91AF10872
:10323000F4CF17FF28C0E0910805F0910905099522
:10324000E0910C05F0910D050995E0911205F091C2
:1032500013050995F6010995E0910A05F0910B0512
:1032600089830995F1E08F1A91088981811491046D
:1032700011F08111E5CFE0910605F0910705099560
:10328000A80CB91C0CC0E0911205F091130509952A
:10329000D6018D936D01B1E08B1A9108A1F7E091F1
:1032A0001205F09113050995E1E0AE1AB108B9F7DE
:1032B0000E94991781E090E0892821F480E002C003
:1032C00084E090E00F90DF91CF911F910F91FF90DC
:1032D000EF90DF90CF90BF90AF909F908F90089528
:1032E0000F931F93E0911605F09117059C01225052
:1032F000310940855185425051092417350768F43A
:10330000A181B0E00E94AB390289138924893589F3
:10331000600F711F821F931F03C060E070E0CB013C
:103320001F910F910895CF93DF93EC01E091160563
:10333000F0911705198218828C819D818130910549
:10334000B9F0208531858217930790F49F838E838F
:10335000009719F00E94701904C0668577858089EE
:103360009189688779878A879B8780E090E002C08F
:1033700081E090E0DF91CF9108958F929F92AF927C
:10338000BF92CF92DF92EF92FF920F931F93CF9352
:10339000DF9300D000D0CDB7DEB77C01C09016051A
:1033A000D09017058230910508F473C0F60180852E
:1033B0009185E816F90608F06CC08081813021F013
:1033C000823009F44CC065C04701969487948E0CF6
:1033D0009F1C94013170892C99248694A12CB12CC6
:1033E000F60182859385A485B585B501A401480FB2
:1033F000591F6A1F7B1F2F3FF1E03F0729F002E0B2
:1034000010E0CE0101961BC001E010E02FEF31E08B
:10341000CE0101960E94C418892BD9F5F601428588
:103420005385648575854F5F5F4F6F4F7F4F480DA4
:10343000591D6A1D7B1D20E030E0CE0102960E94DE
:10344000C418892B31F589819A81E0FE06C024E0F9
:10345000969587952A95E1F71EC09F701CC097012D
:103460003327220F331FEF2CFF24F60142855385AB
:10347000648575854E0D5F1D611D711D02E010E0B4
:10348000CE0101960E94C418892B19F489819A8172
:1034900002C081E090E00F900F900F900F90DF91AD
:1034A000CF911F910F91FF90EF90DF90CF90BF9041
:1034B000AF909F908F900895EF92FF920F931F937C
:1034C000CF93DF93EC01E0901605F090170508818B
:1034D00019810F5F1F4F19F483E090E049C04885C0
:1034E00059856A857B854115510561057105A1F3F3
:1034F000C8018F709927892BA1F54F5F5F4F6F4FE0
:103500007F4F488759876A877B878E819F81F70124
:10351000009731F48481958108171907E8F621C0D6
:10352000218130E021503109A80164E0569547958A
:103530006A95E1F724233523232B99F40E94BD19C2
:103540008230910598F0F701208531858217930725
:1035500018F69F838E830E947019688779878A87FF
:103560009B871983088380E090E002C081E090E0AF
:10357000DF91CF911F910F91FF90EF900895CF921F
:10358000DF92EF92FF920F931F93CF93DF93EC01A3
:103590006A017B0102E010E02EEF31E00E94C418C6
:1035A000892BC1F48881998185359A4AA9F426E34B
:1035B00030E0B701A601CE010E94C418892B41F466
:1035C00081E0288139812634314439F480E005C016
:1035D00081E003C083E001C082E0DF91CF911F91C1
:1035E0000F91FF90EF90DF90CF900895BF92CF9210
:1035F000DF92EF92FF920F931F93CF93DF93EC0133
:103600006B01FB0180818F3219F4FFEFCF1ADF0AC3
:103610001D821C82F6018081803260F4CE010E94FE
:103620009319E0911605F09117050680F781E02DBA
:103630001082B0C0E0E2BE2EEA81FB81DF01CF0143
:103640000B96A817B90711F0BD92FBCF50E080E0B0
:1036500068E071E0780FD601A80FB11D4C9140329F
:10366000D0F04F32C1F04E3209F47AC0561708F04C
:1036700068C04F3708F065C0842F90E0AFE8B1E034
:103680002D91222309F460C0332727FD3095281798
:103690003907B1F756C0552309F453C0C70ED11CE2
:1036A00081E0403208F080E08387CE010E949319C8
:1036B0000097B1F5E0911605F0911705E680F780C7
:1036C000288139812F70332775E0220F331F7A95B7
:1036D000E1F7488559856A857B8500E210E0C701DE
:1036E0000E94C418892B39F5F70180818823D9F00D
:1036F000838583FD10C06A817B81C701DB019B014B
:10370000255F3F4FA217B30781F1FC015191CF0113
:103710004D915417B9F3CE010E945C1A009781F2C3
:1037200083309105B9F5EA81FB818385882331F0E7
:1037300083E090E02FC081E090E02CC084E090E036
:1037400029C085E090E026C08FE9840F8A3108F413
:103750004052DF01A50FB11D4C935F5F872F79CFDA
:10376000683079F758E06BE0F9CFFB018385811170
:103770000FC0E0911605F09117050680F781E02D46
:10378000838584FFDBCF828D938D9D838C8354CF83
:1037900080E090E0DF91CF911F910F91FF90EF902B
:1037A000DF90CF90BF9008954F925F926F927F927B
:1037B000AF92BF92CF92DF92EF92FF920F931F933F
:1037C000CF93DF93CDB7DEB7A8970FB6F894DEBFDF
:1037D0000FBECDBF5C011092170510921605009721
:1037E00009F4D0C00E941C1880FDCFC040E050E01A
:1037F000BA01CE0101960E94BF1A813009F500E19D
:1038000010E02EEB31E040E050E0BA01CE0101962D
:103810000E94C418892B19F081E090E0B8C08D8116
:10382000811103C089E090E0B2C049845A846B845E
:103830007C84B301A201CE0101960E94BF1A03C08D
:10384000412C512C3201833039F38111EBCF04E24A
:1038500010E02DE030E0B301A201CE0101960E94FC
:10386000C418892BC9F62A853B8540E050E0211514
:1038700031054105510521F4288D398D4A8D5B8D27
:10388000AC81B0E00E94BA396DA37EA38FA398A744
:103890000A811B8120E030E0400E511E621E731E23
:1038A000D5011A964D925D926D927C921D97498139
:1038B00011964C931197CD80DE801596DC92CE92B6
:1038C00014978F819885A0E0B0E00097A105B1051D
:1038D00021F48C899D89AE89BF89F4E0D694C79480
:1038E000FA95E1F7E12CF12CBC01CD01601B710BC5
:1038F000820B930B0DA11EA12FA138A5601B710B8C
:10390000820B930B6C197D098E099F09242F30E0DF
:1039100040E050E00E946A392E5F3F4F4F4F5F4FAB
:10392000D50119963C932E931897273FBFE03B078C
:103930004105510540F0273F3F4F4105510508F033
:1039400071CF82E001C081E0D5018C930DA11EA151
:103950002FA138A5400E511E621E731E1E964D9259
:103960005D926D927C9251974C0C5D1C6E1C7F1C7D
:10397000F501428A538A648A758A1282B0921705C9
:10398000A092160580E090E002C082E090E0A89648
:103990000FB6F894DEBF0FBECDBFDF91CF911F9160
:1039A0000F91FF90EF90DF90CF90BF90AF907F90FE
:1039B0006F905F904F9008950F931F93CF93DF9375
:1039C000CDB7DEB7E8970FB6F894DEBF0FBECDBF18
:1039D00000911605109117050115110569F1F801FF
:1039E00012829E012F5F3F4F37832683205E3F4F19
:1039F00038AB2FA7BC01CE018D960E94F61A009716
:103A0000F9F489818823D1F08C8584FD17C08B8DD2
:103A10009C8DF801978F868F8D8D9E8DAF8DB8A16F
:103A2000828F938FA48FB58F168A178A108E118E6E
:103A300081E0828380E003C088E001C083E090E001
:103A4000E8960FB6F894DEBF0FBECDBFDF91CF91E1
:103A50001F910F9108952F923F924F925F926F9214
:103A60007F928F929F92AF92BF92CF92DF92EF920E
:103A7000FF920F931F93CF93DF9300D000D0CDB769
:103A8000DEB789839A837B014A0180911605909164
:103A900017059C838B83FA0111821082009709F429
:103AA000BBC0FC01828180FFBAC0828D938DA48D42
:103AB000B58D46895789608D718D841B950BA60B3A
:103AC000B70BA70160E070E084179507A607B7075A
:103AD00008F47C01A980BA80612CB2E07B2EE1144D
:103AE000F10409F496C0EB81FC8126883788408C6C
:103AF000518CD201C1019170AA27BB27892B8A2B37
:103B00008B2B09F044C0218130E040E050E0C2013D
:103B1000B101A9E09695879577956795AA95D1F714
:103B20000E946A39672B682B692BA9F4EB81FC8111
:103B300023282428252819F4868D978D04C080A178
:103B400091A10E94BD19EB81FC818230910580F02A
:103B500091A380A31382EB81FC8180A191A10E949B
:103B60007019EB81FC81611571058105910511F4D6
:103B7000128258C02381DC01CB01820F911DA11D4F
:103B8000B11D82A393A3A4A3B5A32F5F2383EB81CD
:103B9000FC81268937893170C301821B930B670131
:103BA0008E159F0508F46C01EB81FC81828142A196
:103BB00053A164A175A1860186FF04C010688981A4
:103BC0009A8101C0C5010E94C418009741F0EB81A1
:103BD000FC811282029731F586E090E025C0AC0CA2
:103BE000BD1CEB81FC8186899789A08DB18D8C0DE0
:103BF0009D1DA11DB11D868B978BA08FB18FF401E8
:103C0000808191818C0D9D1D91838083EC18FD082E
:103C100066CF80E090E008C088E090E005C087E0D3
:103C200090E002C081E090E00F900F900F900F9015
:103C3000DF91CF911F910F91FF90EF90DF90CF9088
:103C4000BF90AF909F908F907F906F905F904F90BC
:103C50003F902F9008954F925F926F927F928F9234
:103C60009F92AF92BF92CF92DF92EF92FF920F930B
:103C70001F93CF93DF9300D000D0CDB7DEB79B0169
:103C800000911605109117050115110509F4D0C012
:103C9000D80112964C91129740FFCDC05A964D9183
:103CA0005D916D917C915D9769017C014C155D057D
:103CB0006E057F0510F46A017B01F801468857887C
:103CC000608C718C168A178A108E118EC114D104E3
:103CD000E104F10409F4B2C08180912CA12CB12C33
:103CE00039E0880C991CAA1CBB1C3A95D1F74114E9
:103CF000510461047104C9F1B1E04B1A5108610823
:103D00007108C701B6016150710981099109A501C6
:103D100094010E946A3929833A834B835C83C301EF
:103D2000B201A50194010E946A3989819A81AB810F
:103D3000BC8182179307A407B507B8F08827992795
:103D4000DC0188199909AA09BB0984219521A621BA
:103D5000B721F801868B978BA08FB18FC81AD90A2B
:103D6000EA0AFB0A80A191A128C0D8015E968D9134
:103D70009C915F9791969C938E9390971EC00E9402
:103D8000BD1982309105F8F0F80120853185821740
:103D90009307C8F4F80191A380A346895789608DE1
:103DA000718D480D591D6A1D7B1D468B578B608F89
:103DB000718FC818D908EA08FB088C149D04AE045A
:103DC000BF04E8F204C0D80112961C921FC0F8018B
:103DD00046895789608D718D4C0D5D1D6E1D7F1D4F
:103DE000468B578B608F718F29E0F694E794D794B8
:103DF000C7942A95D1F7C394C3820E9470196115A4
:103E000071058105910529F4F801128281E090E0A5
:103E100017C0DC01CB010197A109B1098C0D911DDF
:103E2000A11DB11DF80182A393A3A4A3B5A306C04D
:103E300088E090E005C087E090E002C080E090E07C
:103E40000F900F900F900F90DF91CF911F910F91D6
:103E5000FF90EF90DF90CF90BF90AF909F908F90AA
:103E60007F906F905F904F9008950F931F93CF9323
:103E7000DF93CDB7DEB7AC970FB6F894DEBF0FBEB9
